:020000040801F1
:10000000B0790120A101010843140108151301086A
:1000100041140108AD0201087D190108000000002B
:10002000000000000000000000000000471401086C
:10003000AF0201080000000045140108491401083E
:10004000BB010108BB010108BB010108BB0101089C
:10005000BB010108BB010108BB010108BB0101088C
:10006000BB010108BB010108BB010108BB0101087C
:10007000BB010108BB010108BB010108BB0101086C
:10008000BB010108BB010108BB010108BB0101085C
:10009000BB010108BB010108BB010108BB0101084C
:1000A000BB010108BB010108BB010108BB0101083C
:1000B000BB010108BB010108BB010108BB0101082C
:1000C000BB010108BB010108BB010108BB0101081C
:1000D000BB0101086519010871190108BB0101087C
:1000E000BB010108BB010108BB010108BB010108FC
:1000F000BB010108BB010108BB010108BB010108EC
:10010000BB010108BB010108BB010108BB010108DB
:1001100021150108BB010108BB010108BB01010851
:10012000BB010108BB010108BB010108BB010108BB
:10013000BB010108BB010108BB010108BB010108AB
:10014000BB010108BB010108BB010108BB0101089B
:10015000BB010108BB010108BB010108BB0101088B
:10016000BB010108BB010108BB010108BB0101087B
:10017000BB010108BB010108BB0101080000000030
:10018000BB010108BB010108DFF810D000F07CF8CA
:1001900000480047E5190108AFF30080B07901205D
:1001A0000648804706480047FEE7FEE7FEE7FEE711
:1001B000FEE7FEE7FEE7FEE7FEE7FEE7CD140108F7
:1001C000890101082DE9F05F0546002092469B4613
:1001D00088460646814640241BE02846414647465D
:1001E000224600F041F853465A46C01A914110D3B6
:1001F00011461846224600F028F82D1A67EB010830
:100200004F4622460120002100F01FF817EB00099D
:100210004E41201EA4F10104DFDC484631462A4647
:100220004346BDE8F09FD2B201E000F8012B491E21
:10023000FBD270470022F6E710B513460A46044683
:100240001946FFF7F0FF204610BD202A04DB203AB4
:1002500000FA02F1002070479140C2F1200320FA19
:1002600003F3194390407047202A04DB203A21FA17
:1002700002F00021704721FA02F3D040C2F12002BF
:100280009140084319467047064C074D06E0E06868
:1002900040F0010394E8070098471034AC42F6D3CD
:1002A000FFF776FFF81A0108181B0108FEE77047F0
:1002B00070470000002229B101291AD002291BD061
:1002C0004FF440720E490B6823F440730B600B68C7
:1002D00013430B600A6822F0F8020A600A680223DE
:1002E00003EBC00002430A60086840F480300860F5
:1002F00070474FF48072E5E74FF40072E2E70000C8
:10030000103C02401348016889050FD5016821F4AB
:1003100000710160016841F400610160016821F42D
:1003200000610160016841F40071016001684905E4
:100330000FD5016821F480610160016841F48051AA
:100340000160016821F480510160016841F480611D
:1003500001607047003C024008490A6822F440727C
:100360000A600A6842F004020A600A684FF48033A7
:1003700043EA002002430A6070470000103C02403C
:10038000064A136823F440731360136813601368FC
:1003900043F001031360017070470000103C0240FD
:1003A000084910B50C6824F440740C600C6844F4DF
:1003B00040740C600C6844F001040C6002604360FF
:1003C00010BD0000103C0240074A136823F440733C
:1003D0001360136843F480731360136843F00103E0
:1003E0001360018070470000103C0240074A136808
:1003F00023F440731360136843F4007313601368AD
:1004000043F001031360016070470000103C02409C
:1004100017490868C206174805D5C26942F010029C
:10042000C26110220A600A68920605D5C26942F0CC
:100430000802C26120220A600A68520605D5C26914
:1004400042F00402C26140220A600A68120605D521
:10045000C26942F00202C26180220A600A68920701
:1004600005D5C26942F02002C261022008607047CF
:100470000C3C02409039012070B51149044600201F
:10048000C86100F0BBF906460E4D09E0601C07D0BC
:1004900024B100F0B3F9801BA04201D9032070BD44
:1004A0002868C003F2D42868C00701D00120286062
:1004B000286810F0F200F2D0FFF7AAFF012070BD0B
:1004C000903901200C3C024090F83510022903D0ED
:1004D0008021416501207047052180F835100068B2
:1004E000016821F001010160002070472DE9F0470B
:1004F000044622480F46017E01290AD00121804688
:1005000001764CF250394846FFF7B6FF020003D09F
:100510002FE00220BDE8F0874FF0FF303860206800
:10052000174D012801D0A6681CE0207C6168FFF708
:1005300013FF4846FFF7A0FF0246286820F004009A
:10054000286014E0217C3046FFF7B4FE4846FFF7F0
:1005500093FF0200286820F0FA00286001D03E6076
:1005600005E0761CD4E902100844B042EAD8FFF74F
:10057000C9FE002188F818101046CBE790390120F9
:10058000103C02400348016841F000410160002036
:1005900070470000103C02402DE9F0471B4E054615
:1005A0001446307E1F468946012808D00120307647
:1005B0004CF250384046FFF75FFF18B114E00220BC
:1005C000BDE8F0879DB1012D16D0022D19D022462D
:1005D0003B464846FFF7E4FE4046FFF74DFF0C4917
:1005E0000A6822F001020A6000213176E8E7E1B2F0
:1005F0004846FFF7C5FEEFE7A1B24846FFF7E4FE25
:10060000EAE721464846FFF7F1FEE5E79039012089
:10061000103C0240074900200A68002A09DA054A0E
:10062000054B0C3A1360054B13600968002900DA8A
:1006300001207047103C024023016745AB89EFCD94
:100640002DE9F84FDFF87CB100224FF001084FF0A0
:10065000030A4FF00F090BF1040E00BF0B6808FAF4
:1006600002F42340A3426ED14D68022D01D0122D19
:100670000ED1D50800EB850CDCF820505607F70E9C
:1006800009FA07F6B5430E69BE402E43CCF8206048
:10069000066855000F790AFA05FC07F0030726EAF9
:1006A0000C06AF40374307604E68012E05D0022E7E
:1006B00003D0112E01D0122E0ED18668CF6826EA03
:1006C0000C06AF40374387604668A6430C79C4F3F5
:1006D0000014944034434460C6688C6826EA0C06D3
:1006E000AC403443C4604C68E40065D5364C2568A2
:1006F00045F480452560246822F0030504F4804415
:100700000094324C2E19D6F8084895072F0F09FA95
:1007100007F5AC432E4DA84201D1002524E02D4D14
:10072000A84201D101251FE02B4DA84201D102258D
:100730001AE02A4DA84201D1032515E0284DA84210
:1007400002D1042510E037E0264DA84201D105254D
:100750000AE0254DA84201D1062505E0234DA84217
:1007600001D1072500E00825BD402543C6F80858FB
:10077000DBF800405D464E689C43F60300D51C4301
:100780002C60DEF8004075464E689C43B60300D5E9
:100790001C432C600B4D08352C684E689C43F602B8
:1007A00000D51C432C60074D0C352C684E689C43CB
:1007B000B60200D51C432C60521C102AFFF44EAF29
:1007C000BDE8F88F003C0140443802400030014051
:1007D000000002400004024000080240000C0240F9
:1007E000001002400014024000180240001C0240A9
:1007F0000AB1816170470904FBE700000148806885
:1008000070470000300000200248816802781144DF
:1008100081607047300000200B4810B5016841F43A
:1008200000710160016841F480610160016841F478
:1008300080710160032000F06FF8002000F006F8DE
:1008400000F024F8002010BD003C024070B50D4DB2
:1008500004464FF47A712878B1FBF0F00A49096830
:10086000B1FBF0F000F0E2FA48B9102C07D20022F8
:100870002146501E00F030F800206C6070BD012051
:1008800070BD0000300000203C0000200A4808B580
:10089000016841F480410160006800F480400090EC
:1008A0000548001F016841F080510160006800F0B8
:1008B0008050009008BD000044380240002809DB49
:1008C00000F01F02012191404009800000F1E0206A
:1008D000C0F8001170470000F0B40E4B1B680C46C6
:1008E000C3F30223C3F10705042D00D90425191D04
:1008F000072901D2002300E0DB1E012606FA05F1DC
:10090000491E214099409E40761E16403143F0BC5E
:1009100001F048B80CED00E0064900F00702086855
:100920004FF6FF03184040EA0220034A10430860D4
:10093000704700000CED00E00000FA052DE9F047DB
:100940000E46050065D0DFF81481D8F80000F7B234
:1009500000F00F00B04207D288F80070D8F800000D
:1009600000F00F00B04254D128683D4C810712D5E9
:10097000400703D5206840F4E05020602878000745
:1009800003D5206840F4604020602068A96820F00A
:10099000F000084320602878C0072DD030496868EF
:1009A0000839012812D0022813D0032811D0096871
:1009B000890700292DDA216821F003010143216014
:1009C000FFF71CFF814641F2883A0EE0096889036F
:1009D000EFE709688901ECE7FFF710FFA0EB0901D9
:1009E000514502D90320BDE8F0872068696800F00E
:1009F0000C00B0EB810FEFD1D8F80010404601F0A9
:100A00000F01B14207D90770006800F00F00B04233
:100A100001D00120E7E72878400705D52068E9687C
:100A200020F4E050084320602878000706D52068AD
:100A3000296920F4604040EAC100206000F036F8E7
:100A40002168084AC1F30311515CC8400649086097
:100A50000020FFF7FBFE0020C5E70000003C02403D
:100A600008380240E01A01083C000020044805490B
:100A700000680968044AC1F38221515CC84070478C
:100A80003C00002008380240F01A010804480549DB
:100A900000680968044AC1F34231515CC84070479C
:100AA0003C00002008380240F01A0108154810B533
:100AB000006810F00C02144813D01449042A0FD017
:100AC000082A0ED10F4C241F2268236802F03F022F
:100AD0005B0207D52068C0F38810A0FB010106E087
:100AE000084610BD2168C1F38811A1FB0001002355
:100AF000FFF768FB2168C1F30141491C4900B0FBC5
:100B0000F1F010BD083802400024F40040787D0167
:100B10002DE9F84F050076D02878DFF8F8B2BE4C02
:100B2000C00749D0DBF800105846C1F38101012904
:100B300008D00068C0F3810002280AD1201D006897
:100B4000400206D52068800336D568680028E2D0C8
:100B500032E06868B0F5803F10D0B0F5A02F206873
:100B600010D020F480302060206820F480202060A5
:100B70006868A0B1FFF742FE06460CE0206840F42A
:100B80008030F4E740F480202060F7E7FFF736FE7E
:100B9000801B642873D820688003F7D50CE0FFF72A
:100BA0002DFE064605E000BFFFF728FE801B6428E7
:100BB000F0D820688003F7D42878DFF860828007B7
:100BC0004FF000093ED5DBF80010584611F00C0F2D
:100BD00009D00068C0F3810002280BD18D48001FA6
:100BE0000068400206D42068800715D5E86801280F
:100BF00009D111E0E868B8B10120C8F80000FFF79A
:100C0000FDFD064605E002E1FFF7F8FD801B022826
:100C1000C0D820688007F7D52068296920F0F8003F
:100C200040EAC10020600DE0C8F80090FFF7E6FD43
:100C3000064604E0FFF7E2FD801B02281FD820686B
:100C40008007F7D42878000722D5724E7448696966
:100C50006C3671B101210160FFF7D0FD074604E059
:100C6000FFF7CCFDC01B022809D830688007F7D5F4
:100C70000EE0C0F80090FFF7C1FD074605E083E0F5
:100C8000FFF7BCFDC01B02287ED830688007F7D470
:100C90002878400768D5DFF87CA100270AF1380AD8
:100CA000DAF80000C0000BD4DAF8001041F08051EF
:100CB000CAF80010DAF80000012700F08050009018
:100CC000584E3068C00510D4306840F480703060F1
:100CD000FFF794FD009005E0FFF790FD0099401AA2
:100CE000022851D83068C005F6D54A4EA868683643
:100CF00001280FD00528306810D020F001003060A6
:100D0000306820F004003060A868B8B1FFF776FDC5
:100D100000900FE0306840F00100F4E740F004007C
:100D20003060F7E7FFF76AFD0099411A41F2883019
:100D3000814264D830688007F4D50EE0FFF75EFD8D
:100D4000009007E0FFF75AFD0099411A41F2883000
:100D5000814254D830688007F4D42FB1DAF80010FB
:100D600021F08051CAF80010A869C0B3DBF8001068
:100D7000C1F3810102294AD00228484607D0C8F8A9
:100D80006000FFF73BFD00E039E005463AE04746EA
:100D9000C8F86000FFF732FD064604E0FFF72EFDBD
:100DA000801B02282BD820688001F7D4D5E90701E1
:100DB0000843A96A1C4A490802EB01416A6A41EAF0
:100DC0008211084395F82C1040EA01611148001F78
:100DD000016001203866FFF711FD054605E014E0CB
:100DE000FFF70CFD401B022809D820688001F7D5C9
:100DF0000BE000BFFFF702FD401B022802D90320D1
:100E0000BDE8F88F20688001F4D40020F8E70120C5
:100E1000F6E7000008380240003802400000474270
:100E2000800E4742007000400000FFFF10B5401EDA
:100E3000B0F1807F01D3012010BD4FF0E02460614C
:100E40000F21601700F0AEFD0020A0610720206197
:100E5000002010BD7047000070B50268044610689D
:100E6000D168536910F00F0F50D003F0010501F461
:100E7000907635435DD0C20705D0CA0503D5E26B35
:100E800042F00102E263420705D5DA0703D0E26BC4
:100E900042F00202E263820705D5DA0703D0E26B73
:100EA00042F00402E263020705D5DA0703D0E26BE1
:100EB00042F00802E263E26B002A33D0800604D5D8
:100EC000880602D5204600F047FB20684069E16BA8
:100ED000C0F38010090700D428B3204600F02EFB91
:100EE0002068416949061AD5416921F040014161F4
:100EF000606BA0B11B490165606BFFF7E5FA002844
:100F000010D0606B016DBDE870400847830610D5B6
:100F10008B060ED52046BDE8704000F01DBB204674
:100F2000FFF798FF70BD2046FFF794FF0020E063B5
:100F300070BD030606D50B0604D52046BDE87040FB
:100F400000F0ACBC4006F3D54806F1D5D168204688
:100F500021F04001D160202184F8391000F0D9F946
:100F600070BD00002D15010870B5040004D094F880
:100F70003900002510B106E0012070BD84F838501A
:100F8000204600F023F8242084F839002068C16846
:100F900021F40051C160204600F02AFB206801695D
:100FA00021F4904101612068416921F02A014161E9
:100FB0002068C16841F40051C160E563202084F8D5
:100FC000390084F83A00002070BD0000F0B587B009
:100FD000044614216846FFF72DF93A48384E256833
:100FE00038491038022201230324B5421FD10D686D
:100FF00045F400250D60096801F4002105910168A0
:1010000041F0040101600068694600F004000590A9
:10101000A0028DE81D00082004902B48FFF710FB6C
:10102000002211463420FFF757FC342022E0274FDE
:101030000726BD4222D12349091D0D6845F0100540
:101040000D60096801F010010591016841F002018D
:1010500001600068694600F002000590C0208DE83C
:101060005D001B48FFF7ECFA002211462520FFF730
:1010700033FC2520FFF722FC07B0F0BD154FBD4221
:10108000FAD10D6845F400350D60096801F40031AE
:101090000591016841F0080101600068694600F0AF
:1010A0000800059060208DE85D000B48FFF7C8FA46
:1010B000002211462620FFF70FFC2620DAE7000069
:1010C000004C00404038024000080240001001403F
:1010D0000004024000440040000C024090F83A3006
:1010E000202B22D1F9B1F2B190F83830012B1CD06D
:1010F00081628285C2850021C163222280F83A2064
:1011000080F838100168CA6842F48072CA600168C9
:101110004A6942F001024A610068C16841F0200159
:10112000C160002070470120704702207047000016
:101130002DE9F0410068424988423AD1414C60684B
:1011400001280AD0002834D104F114052878FF289A
:101150002FD1687801282ED045E0002525613A4A34
:10116000DFF8E8C0A168206902EB800312F8207064
:10117000DE7806EB07665F789B783F0407EB032376
:10118000334400EB8106401C4CF8263020610428D3
:10119000E9DBE068401E814208D100F06FFC00F0FE
:1011A00055FC00F0EDFB6560E560A560A068401CA3
:1011B000A060BDE8F081A8790D28FAD14FF6FF7341
:1011C00001222049224800F047F801206060A978F8
:1011D000E87801EBC10202EB011100EB8100E06055
:1011E0002878FF28E5D168781A4E4FF48044022809
:1011F00011D1A8790D28DCD1012221463046FFF714
:10120000F7FA10490A2307221B31114800F024F88D
:101210002878FF28CDD168780328CAD1A8790D286D
:10122000C7D1002221463046FFF7E2FABDE8F0417F
:1012300004490A2307222231054800F00DB80000B6
:10124000004C004000000020C0380120809C00209D
:10125000D0380120000C02402DE9F843044690F8F4
:1012600039001F4616460D46202850D1A5B19EB123
:1012700094F8380001284AD0012084F838004FF053
:101280000008C4F83C80212084F83900FFF7B6FA42
:10129000A6848146E68426E00120BDE8F883E08C40
:1012A000401EE084A0684B46B0F5805F4FF000021E
:1012B0004FF080012046009703D000F020FBE8B9F2
:1012C0000DE000F01CFBC8B928882168C0F30800B5
:1012D0004860206908B16D1C05E0AD1C03E0216881
:1012E00015F8010B4860E08C0028D8D14B4600224D
:1012F00040212046009700F002FB08B10320CCE714
:10130000202084F8390084F838800020C5E70220C6
:10131000C3E77047FEE7000070B586B01421684649
:10132000FEF788FF1A480024016841F001010160BE
:10133000016801F001010591016841F008010160B7
:10134000016801F008010591016841F004010160A4
:10135000016801F004010591016841F0020101609A
:1013600000680C4E00F002004FF47045059000221A
:1013700029463046FFF73CFA01200095CDE90104EB
:10138000694630460394FFF75BF906B070BD000074
:1013900030380240000C02400C4810B50A49016088
:1013A0004FF4E1314160002181600C22C160C0E94D
:1013B00004128161C161FFF7D7FD002803D0BDE8A9
:1013C0001040FEF775BF10BD004C0040D038012022
:1013D0000C4810B50A4901604FF4E1314160002129
:1013E00081600C22C160C0E904128161C161FFF714
:1013F000BBFD002803D0BDE81040FEF759BF10BD6B
:1014000000100140103901200C4810B50A49016054
:101410004FF416414160002181600C22C160C0E997
:1014200004128161C161FFF79FFD002803D0BDE870
:101430001040FEF73DBF10BD004400405039012070
:10144000FEE7704770477047FFF7DEB930B593B0DD
:1014500030216846FEF7EEFE14210CA8FEF7EAFEE6
:1014600018480025016841F080510160006800F0D3
:10147000805011901448016841F480410160006877
:10148000022400F480401190012003901020049069
:10149000009406940820CDE907504820CDE90904BE
:1014A00003200B906846FFF733FB0CA90F2081E85F
:1014B0003100E002CDE90F0502210CA8FFF73EFA4A
:1014C00013B030BD40380240007000401048016841
:1014D00041F4700101600F48016841F001010160B1
:1014E0000C4A00210832116002680B4B1A4002605E
:1014F000031D0A4A1A60026822F48022026005482D
:101500000C300160024958068039086070470000BD
:1015100088ED00E000380240FFFFF6FE10300024A6
:101520000148FFF799BC0000D038012010B5806B4E
:101530000021C185C184FFF78DFC10BD0168CA6818
:1015400022F49072CA6001684A6922F001024A617D
:10155000202180F83A10704710B590F83A102229EF
:1015600001D0022010BD8168B1F5805F11D0016902
:10157000002901681FD0496801F07F03816A4A1C75
:1015800082620B70C18D491E0904090CC18518D0F7
:101590002BE00269816A002A0268526805D0D2B243
:1015A0000A80816A491C8162ECE7C2F308020A8062
:1015B000816A891CF7E74A68816A4B1C83620A705A
:1015C000E0E70168CA6822F02002CA600168CA68C0
:1015D00022F48072CA6001684A6922F001024A61FD
:1015E000202180F83A10FFF7A3FD002010BD000075
:1015F0002DE9F041044600680169E26821F4405198
:10160000114301612169A068E269084361691143DE
:1016100022680843D16849F20C6399430143D160C1
:1016200020684169A26921F4407111434161E26976
:101630006425B2F5004F9748974922684FF0320869
:101640003FD08A4201D082427CD1FFF71FFA00EBE3
:10165000C00101EB001061688900B0FBF1F6FFF7F3
:1016600015FA00EBC00101EB001061688900B0FBC6
:10167000F1F0B0FBF5F06FF01801484306EB800184
:1016800008EB0110B0FBF5F000F0F006FFF7FEF9F3
:1016900000EBC00101EB001061688900B0FBF1F0C4
:1016A000B0FBF5F006EB0016FFF7F0F900EBC00118
:1016B00001EB001061688900B0FBF1F7FFF7E6F974
:1016C000D2E08A4201D082423DD1FFF7DFF900EB40
:1016D000C00101EB001061684900B0FBF1F0B0FB04
:1016E000F5F00601FFF7D2F900EBC00101EB0010A5
:1016F00061684900B0FBF1F7FFF7C8F900EBC001E2
:1017000001EB001061684900B0FBF1F0B0FBF5F0AF
:101710006FF01801484307EB800108EBC100B0FBF4
:10172000F5F000F0F80006EB4006FFF7AFF900EB2C
:10173000C00101EB001061684900B0FBF1F7FFF751
:10174000A5F93CE055E0FFF791F900EBC00101EB92
:10175000001061684900B0FBF1F0B0FBF5F0060144
:10176000FFF784F900EBC00101EB0010616849004C
:10177000B0FBF1F7FFF77AF900EBC00101EB0010C5
:1017800061684900B0FBF1F0B0FBF5F06FF01801B3
:10179000484307EB800108EBC100B0FBF5F000F017
:1017A000F80006EB4006FFF761F900EBC00101EB22
:1017B000001061684900B0FBF1F7FFF757F900EB43
:1017C000C00101EB001061684900B0FBF1F0B0FB13
:1017D000F5F06FF01801484307EB800108EBC100FA
:1017E000B0FBF5F000F00700216830448860BDE8E8
:1017F000F081FFF73BF900EBC00101EB00106168DD
:101800008900B0FBF1F6FFF731F900EBC00101EB05
:10181000001061688900B0FBF1F0B0FBF5F06FF0EB
:101820001801484306EB800108EB0110B0FBF5F00E
:1018300000F0F006FFF71AF900EBC00101EB001011
:1018400061688900B0FBF1F0B0FBF5F006EB001623
:10185000FFF70CF900EBC00101EB00106168890093
:10186000B0FBF1F7FFF702F900EBC00101EB00104C
:1018700061688900B0FBF1F0B0FBF5F06FF0180182
:10188000484307EB800108EB0110B0FBF5F000F0D6
:101890000F00A9E7001401400010014090F8391032
:1018A000212901D0022070478168B1F5805F016A6B
:1018B0000BD04A1C0262026809785160C18C491E33
:1018C0000904090CC1840ED017E009880268C1F32D
:1018D0000801516001690029016A02D0491C0162B6
:1018E000ECE7891CFBE70168CA6822F08002CA6045
:1018F0000068C16841F04001C160002070472DE9D7
:10190000F041984617460E460446069D1DE0681CA9
:101910001BD02DB1FEF772FFA0EB0800A84214D92E
:101920002068C16821F4D071C1602068416921F04C
:1019300001014161202084F8390084F83A00002038
:1019400084F838000320BDE8F0812068006836EA9A
:10195000000004D00020B842D9D00020F3E70120D5
:10196000F9E700000148FFF777BA000010390120BD
:101970000148FFF771BA000050390120FEE700006E
:1019800006490868064A1040B0F1005F04D1486873
:10199000096881F3088800477047000000000108CB
:1019A0000000FE2F0907090E002804DB00F1E020EB
:1019B00080F80014704700F00F0000F1E02080F87C
:1019C000141D704702E008C8121F08C1002AFAD18E
:1019D00070477047002001E001C1121F002AFBD1AF
:1019E00070470000FEF718FFFFF730FDFFF794FC8B
:1019F000FFF70AFDFFF7D0FCFFF7EAFC0E490D48A0
:101A000008600A2307220D490D48FFF725FC012233
:101A100091030C48FEF7ECFE084C293C606828B1A5
:101A2000094910220648FFF759FBF7E70349072247
:101A30001539F7E70000010808ED00E02900002053
:101A4000D0380120000C0240C038012030B50849D0
:101A50000020084B0861084CCA6804E053F8205085
:101A600044F82050401CB0EB820FF7DB086130BD1A
:101A700000000020000001084000002070B588B080
:101A8000FEF7C8FD022004900420029000250120EA
:101A90000390009506A906956846FEF727FD0D4CB4
:101AA0000E4E25610C4D20690BE000BF55F820203B
:101AB00006EB800100230220FEF76EFD2069401C2A
:101AC0002061E168B0EB810FF0DBFEF75BFD08B051
:101AD00070BD000000000020809C00200000010874
:101AE00000000000000000000102030406070809CE
:101AF0000000000001020304181B01080000002080
:101B000040000000C4190108581B010840000020D3
:101B100070790100D419010879000000000000006C
:101B2000000000000000000000000000FFFF0000B7
:101B300000000DFFFF000000010DFFFF000000028C
:101B40000DFFFF000000030D010000001000000069
:081B5000000000000024F40075
:040000050801018964
:00000001FF
